:100000000C94BB010C94FF010C94FF010C94FF01B4
:100010000C94FF010C94FF010C94FF010C94FF0160
:100020000C94FF010C94FF010C94E20A0C94B40BA5
:100030000C94FF010C94FF010C94FF010C94FF0140
:100040000C94FF010C9432200C94FF010C94FF01DE
:100050000C94FF010C94BD190C94FF010C94FF014A
:100060000C94FF010C94FF010C94FF010C94FF0110
:100070000C94FF010C94FF010C94FF010C94FF0100
:100080000C94FF010C94FF010C94FF010C94FF01F0
:100090000C94FF010C94FF010C94FF010C94FF01E0
:1000A0000C94FF010C94FF010C94FF01210C430CF4
:1000B000310D430C310D880CAB0C310D000D130DBF
:1000C000FF0FFF0F3C103C107F10BD10D612D61250
:1000D000D610D612D711D711AA12D612D612C11223
:1000E00035002B002971E1003A0000001E001400C9
:1000F00004001D003B00E2001F001A0016001B0058
:100100003C00297120000700080006003D002A007D
:100110002100090017001900E300A90022000E00C9
:100120000A0005000000AA003E00310000002F0078
:100130000000A8003F000000000030000000AE00FA
:1001400023000D001C0013000000AB002400180069
:1001500011001000E700AC00250015000C0036006F
:1001600050002C0026000F00120037005100340010
:10017000270033000B0038005200E6002E002D004F
:100180002800E5004F0000001603450072006700DC
:100190006F0044006F007800200045005A00000006
:1001A00016034500720067006F0044006F0078007E
:1001B000200045005A0000000403090409026D00F4
:1001C000040100A0FA090400000103010100092153
:1001D00011010001223F000705810308000A0904FC
:1001E00001000103010200092111010001224D005B
:1001F0000705820308000A09040200010300000049
:100200000921110100012236000705830308000AB5
:10021000090403000103000000092111010001226B
:1002200039000705840310000112011001000000CD
:1002300008EDFE071301000102000105010906A1F6
:1002400001050719E029E7150025019508750181C9
:100250000205081901290595057501910295017599
:100260000391010507190029771500250195787577
:10027000018102C005010980A10185021601002645
:10028000B7001A01002AB700751095018100C0055A
:100290000C0901A1018503160100269C021A010028
:1002A0002A9C02751095018100C005010902A10177
:1002B0000901A10005091901290515002501950568
:1002C000750181029501750381010501093009312C
:1002D0001581257F95027508810609381581257FCE
:1002E000950175088106050C0A38021581257F9550
:1002F0000175088106C0C005010906A1010507199D
:10030000E029E71500250195087501810295017521
:1003100008810105081901290595057501910295C6
:1003200001750391010507190029FF150025FF95A7
:100330000675088100C000000000000000000000F9
:1003400000010204060A0F17202C3A4A5D71879DAE
:10035000B3C7DAE9F5FCFFFCF5E9DAC7B39D8771AD
:100360005D4A3A2C20170F0A060402010000000023
:1003700000000000000011241FBECFEFDAE0DEBF56
:10038000CDBF04B603FE24C08091EF019091F0012F
:10039000A091F101B091F2018730904BA740B04B92
:1003A000B9F41092EF011092F0011092F101109245
:1003B000F20114BE84B7877F84BF88E10FB6F8943A
:1003C00080936000109260000FBEE0E0FFE30995AB
:1003D00011E0A0E0B1E0E8EEF3E402C005900D9278
:1003E000A433B107D9F711E0A4E3B1E001C01D9235
:1003F000AF3EB107E1F70E9426080C94F2210C945D
:100400000000089556985E9825982D9826982E9865
:1004100027982F98089508950C940B0256985E988B
:1004200025982D9826982E9827982F988FEF90E052
:10043000909389008093880090938B0080938A002A
:1004400090938D0080938C00259A2D9A2FEF80E752
:1004500092E0215080409040E1F700C00000269AD1
:100460002E9A2FEF80E792E0215080409040E1F7F4
:1004700000C00000279A2F9A2FEF80E792E02150CA
:1004800080409040E1F700C0000025982D982FEFA4
:1004900080E792E0215080409040E1F700C00000EA
:1004A00026982E982FEF80E792E0215080409040D0
:1004B000E1F700C0000027982F9856985E9825987D
:1004C0002D9826982E9827982F98089589EA80933A
:1004D000800089E08093810024982C983F988AB10D
:1004E0008F748AB96E98479A8BB1806B8BB9769A64
:1004F0000E940E020C94020280E28093000180911F
:10050000340181110EC00E94CB0281E0809334013E
:100510002FEF83ED90E3215080409040E1F700C041
:10052000000080E40E94D1028093000181112EC05E
:100530000E94FB0280930001811128C00E94FB02EF
:1005400080930001811122C08FE30E94FB028093FF
:10055000000181111BC00E94F30280E40E94D102BD
:1005600080930001811112C08CE00E94FB028093F5
:10057000000181110BC00E94FB02809300018111D8
:1005800005C08FE30E94FB02809300010E94F302EA
:100590008091000108951092B9008AE08093B8001C
:1005A000089594EA9093BC009091BC0097FFFCCF13
:1005B0009091B900987F983021F0903111F081E04E
:1005C00008958093BB0084E88093BC008091BC00B8
:1005D00087FFFCCF8091B900887F883111F080348B
:1005E00071F780E0089584E98093BC008091BC009D
:1005F00084FDFCCF08958093BB0084E88093BC0009
:100600008091BC0087FFFCCF9091B900987F81E07A
:10061000983209F480E0089584E88093BC008091CA
:10062000BC0087FFFCCF8091BB0008958091000142
:10063000811115C080E40E94D102809300018111D4
:100640000CC082E10E94FB0280930001811105C071
:100650008FEF0E94FB02809300010E94F30284B19D
:10066000807F84B985B1807F85B98AB1837F8AB95B
:100670008BB1837F8BB93E98469808950E947C0287
:10068000809300010E94160380B38C7080BB81B3FD
:10069000836F81BBA6E3B1E0E4E4F1E08EE08E0F6E
:1006A00011921D928E13FCCF0C946602BF92CF92D2
:1006B000DF92EF92FF920F931F93CF93DF9380917E
:1006C0000001882379F0809135018F5F8093350197
:1006D000811108C00E947C0280930001811102C038
:1006E0000E940E0206E311E0C0E0D0E0DD24D394C6
:1006F00082E0C82EEE24E394F12CC730D10500F53A
:1007000080910001811164C080E40E94D102809335
:100710000001811112C082E10E94FB02809300015E
:1007200081110BC0C7010C2E01C0880F0A94EAF793
:1007300080950E94FB02809300010E94F30248C052
:10074000CA30A1F028F4C83059F0C93061F005C0B2
:10075000CC3089F070F0CD3089F0209A289810C004
:10076000219A29980DC0229A2A980AC0239A2B9878
:1007700007C0529A01C0539A5B9802C03E9A4698AD
:1007800090EA9A95F1F79FB1799902C082E001C091
:1007900080E091709D25982B7C9902C084E001C077
:1007A00080E0892B7D9902C038E001C030E0832BC6
:1007B0007E9902C020E101C020E0822B9FB190957C
:1007C000991F9927991F9295990F907E892B0FC099
:1007D00080910001811149C080E40E94D102809380
:1007E0000001882379F1B12C0E94F3028B2DF801CE
:1007F0009081981719F08083C09201010E9416031E
:1008000021960F5F1F4FCE30D10509F076CF809132
:100810000101882361F1815080930101882339F01F
:100820008FE99FE00197F1F700C0000020C0A4E429
:10083000B1E0E6E3F1E0CF01825F91919D938E13E9
:10084000FCCF15C083E10E94FB028093000181115F
:10085000CACF81E40E94D102809300018111C3CFED
:100860000E940C03B82EB094BFCF80E0C0CF0E948E
:100870000C0281E0DF91CF911F910F91FF90EF90DB
:10088000DF90CF90BF900895E82FF0E0EC5BFE4F33
:100890008081089508958B3B910578F4883A9105FD
:1008A00040F5853A9105D0F48430910508F0B1C047
:1008B0008130910509F4ADC06BC0803E910508F40C
:1008C00067C0883E910508F4A4C09C01205F3109EF
:1008D0002031310508F05CC090650895853A910596
:1008E00009F459C0863A910509F058C082E890E4AD
:1008F0000895883A910509F454C0893A910509F49C
:1009000053C08A3A910509F452C08B3A910509F413
:1009100051C08C3A910509F450C08D3A910509F403
:100920004FC0803B910509F44EC08E3A910509F401
:100930004DC08F3A910509F44CC0813B910509F4F3
:100940004BC0823B910509F44AC0833B910509F4F1
:1009500049C0843B910509F448C0853B910509F4E1
:1009600047C0863B910509F446C0873B910509F4D1
:1009700045C0883B910509F444C0893B910509F4C1
:1009800043C08A3B910509F442C080E094E4089595
:1009900080E090E0089581E890E4089583E890E491
:1009A000089582EE94E4089589EE94E408958AEE21
:1009B00094E4089585EB94E4089586EB94E4089517
:1009C00087EB94E408958CEC94E408958DEC94E422
:1009D000089583E895E408958AE895E4089582E906
:1009E00095E4089584E995E4089581E296E40895F4
:1009F00083E296E4089584E296E4089585E296E41D
:100A0000089586E296E4089587E296E408958AE2DE
:100A100096E40895089596E0799FF001112494E5F5
:100A2000899FE00DF11D1124E60FF11DEE0FFF1F50
:100A3000E052FF4F859194910895880F991FFC0112
:100A4000E05AF040859194910895880F991FFC0118
:100A5000E052FF4F85919491089526E0729FF00136
:100A6000112444E5849FE00DF11D1124E60FF11DD2
:100A7000EE0FFF1FE052FF4F859194919C013A9534
:100A800021154FE1340708F41CC13F5121153041B5
:100A900020F49F700E94250508959C013053211574
:100AA000304118F49927906C0895811520E592073C
:100AB00071F40E94FA124FEF84E39CE041508040B1
:100AC0009040E1F700C000000E94E219FAC08130B6
:100AD00020E5920731F48091CD0181608093CD01B2
:100AE000F0C09C0130552115304108F051C0292F2C
:100AF00033272F70332721303105D9F4AC014370EF
:100B0000552702C0220F331F4A95E2F73C68AC011B
:100B100064E0440F551F6A95E1F744275370242B76
:100B2000352B73E0880F991F7A95E1F78076992726
:100B30001DC02230310529F4982F8827816F906AD3
:100B4000089523303105A9F4AC014370552721E005
:100B500030E002C0220F331F4A95E2F73C6843E0C1
:100B6000880F991F4A95E1F7807E9770822B932B0F
:100B7000089524303105E1F4AC014370552721E09C
:100B800030E002C0220F331F4A95E2F73A68E7CF00
:100B90009C0130572115304118F49F7090620895E0
:100BA0009C0130582115304118F49F70906A0895C7
:100BB000803E9105E0F4803C910558F58133910524
:100BC00009F46FC048F48932910509F463C08A3290
:100BD000910509F46DC072C089339105E9F082383E
:100BE0009105D1F08533910509F44DC067C0833E6E
:100BF000910581F138F4803E9105B9F0823E91056E
:100C0000D9F05CC0863E910561F1873E9105A1F166
:100C100055C00E941D0508952091E00120FD02C0ED
:100C200021FF4CC080EE90E049C08091E00180FF40
:100C3000F9CF89E390E042C08091E00182FF0EC0CD
:100C40008091E00184FF03C080E090E037C083EE34
:100C500090E034C08091E00182FFF2CF82EE90E01C
:100C60002DC08091E00183FF0BC08091E00184FDE5
:100C7000EBCF87EE90E022C08091E00183FFF5CFBB
:100C800086EE90E01BC08091E00185FF07C089E2FD
:100C900090E014C08091E00185FFF9CF85E390E0FA
:100CA0000DC08091E00186FF07C08AE290E006C097
:100CB0008091E00186FFF9CF81E390E00E944B0430
:100CC0000895089508950C94620680916201089534
:100CD000CF93DF9300D01F92CDB7DEB79C018091F8
:100CE000E601843019F593E099833B832A8390933E
:100CF000E9008FEF9091E800815095FD06C095EDD9
:100D00009A95F1F700008111F5CF8091E80085FFF9
:100D10000DC040E050E063E070E0CE0101960E941B
:100D2000D2088091E8008E778093E8000F900F90B2
:100D30000F90DF91CF910895CF93DF9300D01F9252
:100D4000CDB7DEB72091E601243021F522E02983DA
:100D50009B838A8383E08093E9008FEF9091E80082
:100D6000815095FD06C095ED9A95F1F7000081112F
:100D7000F5CF8091E80085FF0DC040E050E063E0D2
:100D800070E0CE0101960E94D2088091E8008E7733
:100D90008093E8000F900F900F90DF91CF9108950E
:100DA0002091E6012430F1F422E02093E9002FEFB6
:100DB0003091E800215035FD06C035ED3A95F1F748
:100DC00000002111F5CF2091E80025FF0BC040E085
:100DD00050E065E070E00E94D2088091E8008E77D4
:100DE0008093E8000895CF93DF93EC019091E601A2
:100DF000943009F046C080910C018823D9F080918D
:100E00000D018823B9F09093E9008FEF9091E800ED
:100E1000815095FD06C095E19A95F1F7000081118A
:100E2000F5CF8091E80085FF2CC040E050E060E104
:100E300070E017C081E08093E9008FEF9091E800A7
:100E4000815095FD06C095ED9A95F1F7000081114E
:100E5000F5CF8091E80085FF14C040E050E068E0E5
:100E600070E0CE010E94D2088091E8008E778093D6
:100E7000E80080E1FE01A2E5B1E001900D928A95C3
:100E8000E1F7DF91CF9108958091E501811109C0CB
:100E90000E94670A0E94C40A8091E20084608093E5
:100EA000E20008951092E501089508950C941F2022
:100EB0000E9478190E9425200E946A0D0C946306F6
:100EC00042E061EC81E00E94E10942E061EC82E0F5
:100ED0000E94E10942E061EC83E00E94E10942E105
:100EE00061EC84E00C94E1098091E801833009F41D
:100EF00055C030F4813071F0823009F48EC008950D
:100F00008A3009F47AC08B3009F460C0893009F066
:100F10009CC020C08091E701813A09F096C0809181
:100F2000E800877F8093E8008091EB019091EC01CD
:100F3000892B21F460E182E591E003C060E080E06C
:100F400090E070E00E941D098091E8008B7780930B
:100F5000E80008958091E701813209F076C0809120
:100F6000EB019091EC01009719F0039709F06DC027
:100F70008091E800877F8093E8008091E80082FDFF
:100F800005C08091E6018111F8CF5FC08091F1002A
:100F9000809362018091E8008B7753C08091E701D4
:100FA000813A09F052C08091EB019091EC01892BBC
:100FB00009F04BC08091E800877F8093E800809122
:100FC000E80080FFFCCF80910C0136C08091E701E2
:100FD0008132D9F58091EB019091EC01892BA9F533
:100FE0008091E800877F8093E8000E94160A809134
:100FF000E90180930C010C94FA128091E70181328F
:1010000021F58091E800877F8093E8000E94160A0E
:101010008091EA018093630108958091E701813A0C
:10102000A1F48091E800877F8093E8008091E80038
:1010300080FFFCCF809163018093F1008091E800F4
:101040008E778093E8000C94160A089584B7877F02
:1010500084BF88E10FB6F89480936000109260001E
:101060000FBE90E080E80FB6F894809361009093F3
:1010700061000FBE0E94B90D0E94670A0E94C40A57
:101080008091E20084608093E20078940E944A0D8F
:101090000E94BB0D82E091E00E94650D0E940D2030
:1010A0008091E601853069F40E9439198091E4014C
:1010B0008823B1F30E946419882391F30E94BC082D
:1010C000EFCF0E94C10DECCF292F332723303105FC
:1010D000C9F064F42130310581F02230310509F086
:1010E00043C08DE690E02CEB31E042C02132310567
:1010F000F1F02232310541F137C082E190E029E27E
:1011000032E036C099278130910541F08230910557
:1011100041F0892B49F5E8EBF1E005C0E0EAF1E0A8
:1011200002C0E8E8F1E0849190E09F0121C06430C2
:10113000D8F4E62FF0E0EE0FFF1FEE5DFE4F2081AA
:10114000318189E090E014C0643070F470E0FB01FC
:10115000EE0FFF1FE65EFE4F20813181FB01EA5E4C
:10116000FE4F808190E004C080E090E020E030E01D
:10117000FA0131832083089580E189BD82E189BD30
:1011800009B400FEFDCF8091D8008F7D8093D800F8
:101190008091E00082608093E0008091E00081FD1A
:1011A000FCCF0895CF92DF92EF92FF920F931F939F
:1011B000CF93DF93EC018B016A010E94350A811104
:1011C00033C0C114D10439F0F60180819181081B2C
:1011D000190BC80FD91FE12CF12C0115110519F1BC
:1011E0008091E80085FD16C08091E8008E7780939D
:1011F000E800C114D10449F0F60180819181E80E24
:10120000F91EF182E08285E00FC00E94350A882332
:1012100021F30AC089918093F10001501109FFEF79
:10122000EF1AFF0ADACF80E0DF91CF911F910F9183
:10123000FF90EF90DF90CF9008952091ED013091D5
:10124000EE012617370748F06115710539F4209132
:10125000E8002E772093E80001C0B90140E0611555
:101260007105A9F12091E601222309F443C025303C
:1012700009F442C02091E80023FD40C02091E8001D
:1012800022FD32C02091E80020FFE9CF4091F30019
:101290002091F20030E0342BFC01CF016115710583
:1012A00059F02830310540F481918093F10061506C
:1012B00071092F5F3F4FF1CF41E02830310509F030
:1012C00040E02091E8002E772093E800C8CF41113C
:1012D000C9CF0AC08091E601882361F0853061F0B2
:1012E0008091E80083FD0AC08091E80082FFF2CF80
:1012F00080E0089582E0089583E0089581E00895F4
:101300002091ED013091EE012617370748F0611565
:10131000710539F42091E8002E772093E80001C090
:10132000B901FC0120E06115710591F18091E601A0
:10133000882309F440C0853009F43FC08091E8005B
:1013400083FD3DC08091E80082FD2FC08091E800C0
:1013500080FFE9CF2091F3008091F20090E0922B82
:101360006115710559F08830910540F4249120935E
:10137000F1003196615071090196F2CF21E0089792
:1013800009F020E08091E8008E778093E800CBCFD1
:101390002111CCCF0AC08091E601882361F085300D
:1013A00061F08091E80083FD0AC08091E80082FF2F
:1013B000F2CF80E0089582E0089583E0089581E00F
:1013C0000895982F973058F59093E900981739F0C1
:1013D0007091EC002091ED005091F00003C0242F9B
:1013E000762F50E021FF19C03091EB003E7F309303
:1013F000EB003091ED003D7F3093ED003091EB003C
:1014000031603093EB007093EC002093ED0050932B
:10141000F0002091EE0027FF07C09F5FD3CF8F70B1
:101420008093E90081E0089580E008958091E701CC
:1014300087FF11C08091E80082FD05C08091E60120
:101440008111F8CF11C08091E8008B770BC080919B
:10145000E601882349F08091E80080FFF8CF809171
:10146000E8008E778093E80008952091E4003091A1
:10147000E50095E64091EC00842F817040FF22C08A
:101480008091E80080FD1CC08091E601882391F0E6
:10149000853091F08091EB0085FD10C04091E40013
:1014A0005091E5004217530729F39A01915011F723
:1014B00084E0089582E0089583E0089581E008952E
:1014C00080E008954091E80042FFDECF08950E9439
:1014D000D50A0E94DD0AE0EEF0E080818160808321
:1014E000E8EDF0E080818F77808319BCA7EDB0E054
:1014F0008C918E7F8C9380818F7E80831092E5010A
:1015000008950F931F93CF93DF930E94D50A0E94F3
:10151000DD0AC8EDD0E088818F7788838881806874
:10152000888388818F7D888319BC1092E601109290
:10153000E2011092E4011092E30100EE10E0F801E4
:1015400080818B7F808388818160888342E060E036
:1015500080E00E94E109E1EEF0E080818E7F8083EF
:10156000E2EEF0E08081816080838081886080830A
:10157000F80180818E7F8083888180618883DF91FC
:10158000CF911F910F910895E8EDF0E080818F7E5B
:101590008083E7EDF0E080818160808384E082BF1A
:1015A00081E08093E5010C94810AE8EDF0E0808110
:1015B0008E7F80831092E20008951092DA001092DC
:1015C000E10008951F920F920FB60F9211242F93EE
:1015D0003F934F935F936F937F938F939F93AF93BB
:1015E000BF93EF93FF938091E10082FF0BC0809146
:1015F000E20082FF07C08091E1008B7F8093E100D1
:101600000E94490D8091DA0080FF1FC08091D800B0
:1016100080FF1BC08091DA008E7F8093DA0080917A
:10162000D90080FF0DC080E189BD82E189BD09B488
:1016300000FEFDCF81E08093E6010E94440705C0D3
:1016400019BC1092E6010E9452078091E10080FFD0
:1016500019C08091E20080FF15C08091E2008E7F6A
:101660008093E2008091E20080618093E2008091AB
:10167000D80080628093D80019BC85E08093E60191
:101680000E9456078091E10084FF30C08091E20003
:1016900084FF2CC080E189BD82E189BD09B400FED0
:1016A000FDCF8091D8008F7D8093D8008091E1009C
:1016B0008F7E8093E1008091E2008F7E8093E20034
:1016C0008091E20081608093E2008091E2018823B2
:1016D00011F084E007C08091E30087FD02C081E043
:1016E00001C083E08093E6010E9458078091E100E9
:1016F00083FF29C08091E20083FF25C08091E10033
:10170000877F8093E10082E08093E6011092E201FE
:101710008091E1008E7F8093E1008091E2008E7FD6
:101720008093E2008091E20080618093E20042E0D9
:1017300060E080E00E94E1098091F0008860809381
:10174000F0000E945507FF91EF91BF91AF919F91DB
:101750008F917F916F915F914F913F912F910F905A
:101760000FBE0F901F9018951F920F920FB60F92F9
:1017700011242F933F934F935F936F937F938F9396
:101780009F93AF93BF93CF93DF93EF93FF93C0915A
:10179000E900CF708091EC00D82FD17080FDD0E8A7
:1017A0001092E9008091F000877F8093F000789498
:1017B0000E94F80B1092E9008091F00088608093FD
:1017C000F000CD2BCF70C093E900FF91EF91DF9136
:1017D000CF91BF91AF919F918F917F916F915F91C9
:1017E0004F913F912F910F900FBE0F901F90189522
:1017F0001F93CF93DF93CDB7DEB7AA970FB6F894B8
:10180000DEBF0FBECDBFE7EEF1E088E08E0F909116
:10181000F10091938E13FBCF0E9474078091E80032
:1018200083FF1FC18091E7019091E801492F50E0AB
:101830004A30510508F015C1FA01EA5AFF4F0C94DD
:10184000A721803881F0823809F00BC18091EB012B
:101850008F708093E9008091EB0085FB882780F9E9
:101860001092E90006C08091E3019091E40191118A
:1018700082609091E800977F9093E8008093F10058
:101880001092F100C8C0282F2D7F09F0EAC08823EC
:1018900019F0823061F0E5C08091E901813009F0F2
:1018A000E0C0933009F080E08093E4012BC0809188
:1018B000E901811127C08091EB018F7009F4D1C03B
:1018C0008093E9002091EB0020FF1CC0933021F4AD
:1018D0008091EB00806214C09091EB009061909336
:1018E000EB0021E030E0A90102C0440F551F8A95AA
:1018F000E2F74093EA001092EA008091EB008860E2
:101900008093EB001092E9008091E800877F86C009
:101910008111A7C01091E9011F778091E3008078C1
:10192000812B8093E3008091E800877F8093E8001B
:101930000E94160A8091E80080FFFCCF8091E300AE
:1019400080688093E300111102C082E001C083E04F
:101950008093E60186C08058823008F082C0809172
:10196000E9019091EA018C3D53E0950779F583E018
:101970008A838AE289834FB7F894DE01139620E0C8
:101980003EE051E2E32FF0E050935700E49120FF56
:1019900003C0E295EF703F5FEF708E2F90E0EA306A
:1019A00010F0C79601C0C0968D939D932F5F243190
:1019B00049F74FBF8091E800877F8093E8006AE293
:1019C00070E0CE0101960E941D0914C0AE014F5F68
:1019D0005F4F6091EB010E946408BC01892B09F400
:1019E00040C09091E800977F9093E80089819A81A8
:1019F0000E9480098091E8008B778093E80031C0D5
:101A0000803879F58091E800877F8093E8008091A5
:101A1000E2018093F1008091E8008E778093E800E6
:101A20000E94160A1EC081111CC09091E9019230DB
:101A3000C0F48091E800877F8093E8009093E201F2
:101A40000E94160A8091E201811106C08091E30094
:101A500087FD02C081E001C084E08093E6010E941E
:101A600060078091E80083FF0AC08091E800877FCB
:101A70008093E8008091EB0080628093EB00AA964F
:101A80000FB6F894DEBF0FBECDBFDF91CF911F918F
:101A900008950895CF938091E6018823A1F0C09125
:101AA000E900CF709091EC00892F817090FD80E863
:101AB000C82B1092E9008091E80083FD0E94F80B8A
:101AC000CF70C093E900CF910895909369018093FE
:101AD00068010895E0916801F0916901309721F063
:101AE0000190F081E02D099480E00895E091680173
:101AF000F0916901309721F00280F381E02D099483
:101B00000895E0916801F0916901309721F0048017
:101B1000F581E02D099408952091660130916701C7
:101B20008217930771F09093670180936601E091AB
:101B30006801F0916901309721F00680F781E02D6E
:101B400009940895209164013091650182179307EB
:101B500071F09093650180936401E0916801F091C8
:101B60006901309721F00084F185E02D09940895F2
:101B700008950C94B80D0E947E190E943E030C94A7
:101B8000441ACF92DF92EF92FF920F931F93CF935D
:101B9000DF93CDB7DEB72B970FB6F894DEBF0FBE3D
:101BA000CDBF0E9456038BE6C82E81E0D82E00E000
:101BB00010E0E02E802F0E944404F60141916F0155
:101BC000F42EF826B1F40F5F1F4F0E30110589F780
:101BD0008FEF89838A831B820E9487198160782F07
:101BE0009D838C8349815A816B818D810E94640E13
:101BF00040C09091CD0191FF04C08B870E944A04A0
:101C00008B8520E030E04F2D50E0922FBA01022E5C
:101C100002C0759567950A94E2F760FF24C02E8391
:101C2000EF8221E030E0690102C0CC0CDD1C9A9506
:101C3000E2F790E08C219D21892B09F420E0288790
:101C40000E9487198160782F9A8789874E815F81EA
:101C500068858A850E94640EF801E559FE4F8081EF
:101C6000C826C08206C02F5F3F4F2630310569F677
:101C7000AACF0E942B1D10916A010E946A0D1817AD
:101C8000A1F00E946A0D80936A012B960FB6F8941A
:101C9000DEBF0FBECDBFDF91CF911F910F91FF909F
:101CA000EF90DF90CF900C9463062B960FB6F894CC
:101CB000DEBF0FBECDBFDF91CF911F910F91FF907F
:101CC000EF90DF90CF900895CF93DF93CDB7DEB73D
:101CD0002B970FB6F894DEBF0FBECDBF4F8358874A
:101CE00069877A878B87DE01119686E0FD01119264
:101CF0008A95E9F785E0FE01379601900D928A9565
:101D0000E1F749815A816B817C818D819E810E949E
:101D100094152B960FB6F894DEBF0FBECDBFDF91A2
:101D2000CF9108950895CF93882309F4C2C0C82F96
:101D3000823859F40E946A0D81FDBBC089E30E947C
:101D40003D180E940A1989E30CC0833879F40E9477
:101D50006A0D80FDAEC083E50E943D180E940A19FD
:101D600083E50E947F18CF910C940A19843859F4A6
:101D70000E946A0D82FD9DC087E40E943D180E946A
:101D80000A1987E4EECF8CEF8C0F813A48F48C2F40
:101D90000E94721F81118DC08C2F0E943D18E3CFCD
:101DA00080E28C0F883048F4C77081E001C0880F52
:101DB000CA95EAF70E94C318D6CF8BE58C0F833003
:101DC00078F4C53A29F0C63A31F083E890E005C0CE
:101DD00081E890E002C082E890E0CF910C948C0DF5
:101DE00088E58C0F833108F064C0C83A39F1C93AEC
:101DF00041F1CA3A49F1CB3A51F1CC3A59F1CD3AD5
:101E000061F1C03B69F1CE3A71F1CF3A79F1C13B52
:101E100081F1C23B89F1C33B91F1C43B99F1C53BD0
:101E2000A1F1C63BA9F1C73BB1F1C83BB9F1C93B30
:101E3000C1F1CA3BC9F180E090E038C082EE90E089
:101E400035C089EE90E032C08AEE90E02FC085EB7D
:101E500090E02CC086EB90E029C087EB90E026C094
:101E60008CEC90E023C08DEC90E020C083E891E002
:101E70001DC08AE891E01AC082E991E017C084E9A8
:101E800091E014C081E292E011C083E292E00EC0C2
:101E900084E292E00BC085E292E008C086E292E024
:101EA00005C087E292E002C08AE292E0CF910C94F2
:101EB000A20DCF910895882309F44BC0823859F4BC
:101EC0000E946A0D81FF45C089E30E943D180E946F
:101ED0000A1989E30CC0833871F40E946A0D80FFEF
:101EE00038C083E50E943D180E940A1983E50E94CC
:101EF0007F180C940A19843859F40E946A0D82FFE5
:101F000028C087E40E943D180E940A1987E4EFCF99
:101F10009CEF980F913A58F390E2980F983050F454
:101F2000877091E001C0990F8A95EAF7892F0E9486
:101F3000C918DFCF9BE5980F933020F480E090E044
:101F40000C948C0D885A833120F480E090E00C943E
:101F5000A20D0895882321F00E94C3180C940A1939
:101F60000895882321F00E94C9180C940A19089535
:101F7000BF92CF92DF92EF92FF920F931F93CF9376
:101F8000DF9300D000D000D0CDB7DEB725E0FC0154
:101F9000DE01119601900D922A95E1F7FC01D080A7
:101FA00011810281258122952F7043815481452B17
:101FB00009F4FCC21F3F21F4FFEFDF1609F4F6C25B
:101FC0007C012E830E94920ED9821A8369817A81C4
:101FD000802F0E943918182FB92E0E94EE170E94E8
:101FE000B5162E81002319F00E94E0182E81EB2DEA
:101FF000E295EF70F0E0E05AFF4F0C94A7218B2D93
:10200000807F9B2D9F70F92E882319F0F29480EF2A
:10201000F822002389F0FF2009F475C280E2810FC5
:10202000883020F48F2D0E94C31803C08F2D0E948A
:10203000D3180E940A1967C2812F0E945B0FFF20EC
:1020400009F4B4C2105E8F2D183018F40E94C9181C
:1020500002C00E94D91826960FB6F894DEBF0FBEB4
:10206000CDBFDF91CF911F910F91FF90EF90DF9047
:10207000CF90BF900C940A193B2D307F8B2D8F7021
:10208000303211F08295807F112319F0113021F147
:102090002CC00023B9F0222309F4A0C1213009F09B
:1020A0009DC126960FB6F894DEBF0FBECDBFDF915F
:1020B000CF911F910F91FF90EF90DF90CF90BF9045
:1020C0000C94F318222319F0213009F46FC28E8387
:1020D0000E94F6188E8196C1002321F0223008F06C
:1020E00065C27CC1211162C28DC1002321F022236F
:1020F00009F474C108C2222309F484C119C22B2D2A
:1021000026952695237030E02115310521F02130E8
:102110003105D1F04BC2002321F0812F9B2D93700C
:1021200002C080E090E026960FB6F894DEBF0FBEA6
:10213000CDBFDF91CF911F910F91FF90EF90DF9076
:10214000CF90BF900C948C0D002321F0812F9B2DFC
:10215000937002C080E090E026960FB6F894DEBF40
:102160000FBECDBFDF91CF911F910F91FF90EF90E8
:10217000DF90CF90BF900C94A20D812F002319F017
:102180000E94331C02C00E949B1C26960FB6F89436
:10219000DEBF0FBECDBFDF91CF911F910F91FF909A
:1021A000EF90DF90CF90BF900C94201D8B2D83700B
:1021B00009F07BC00111FAC1812F82958695877045
:1021C000880F880F912F9F70C92ED12CE12CF12CF4
:1021D000082E04C0CC0CDD1CEE1CFF1C0A94D2F7A8
:1021E00014FF12C04FE050E060E070E004C0440F04
:1021F000551F661F771F8A95D2F7CB01BA016095EC
:1022000070958095909503C060E070E0CB012B2D18
:10221000269526952370422F50E042305105D9F083
:102220004330510569F16C297D298E299F29413060
:10223000510551F126960FB6F894DEBF0FBECDBF03
:10224000DF91CF911F910F91FF90EF90DF90CF9092
:10225000BF900C94DC166C297D298E299F29269627
:102260000FB6F894DEBF0FBECDBFDF91CF911F91A7
:102270000F91FF90EF90DF90CF90BF900C94F816E5
:102280000E94DC16C701B60126960FB6F894DEBF91
:102290000FBECDBFDF91CF911F910F91FF90EF90B7
:1022A000DF90CF90BF900C94C016002319F08B2DB7
:1022B000817001C08695882309F478C1812F8295A9
:1022C00086958770880F880F912F9F70C92ED12C0B
:1022D000E12CF12C082E04C0CC0CDD1CEE1CFF1CE4
:1022E0000A94D2F714FF12C04FE050E060E070E0B3
:1022F00004C0440F551F661F771F8A95D2F7CB0184
:10230000BA01609570958095909503C060E070E08B
:10231000CB012B2D269526952370422F50E042307D
:102320005105D9F04330510569F16C297D298E2979
:102330009F294130510551F126960FB6F894DEBF22
:102340000FBECDBFDF91CF911F910F91FF90EF9006
:10235000DF90CF90BF900C94B6176C297D298E2901
:102360009F2926960FB6F894DEBF0FBECDBFDF9132
:10237000CF911F910F91FF90EF90DF90CF90BF9082
:102380000C94D2170E94B617C701B60126960FB655
:10239000F894DEBF0FBECDBFDF91CF911F910F919B
:1023A000FF90EF90DF90CF90BF900C949A17103F62
:1023B000D1F118F4103E50F4A1C0123F09F463C0EB
:1023C00008F44CC0133F09F473C098C01F708B2DE4
:1023D0008F710023A1F00E943317812F26960FB62C
:1023E000F894DEBF0FBECDBFDF91CF911F910F914B
:1023F000FF90EF90DF90CF90BF900C94AA0F0E94B7
:102400005417812F26960FB6F894DEBF0FBECDBFAE
:10241000DF91CF911F910F91FF90EF90DF90CF90C0
:10242000BF900C94B10F0023A9F02111BFC08B2DD8
:102430008F7126960FB6F894DEBF0FBECDBFDF9129
:10244000CF911F910F91FF90EF90DF90CF90BF90B1
:102450000C947917223008F0A9C0E9CF0023A9F025
:102460008B2D8F7126960FB6F894DEBF0FBECDBFB1
:10247000DF91CF911F910F91FF90EF90DF90CF9060
:10248000BF900C943317002359F38B2D8F71269630
:102490000FB6F894DEBF0FBECDBFDF91CF911F9175
:1024A0000F91FF90EF90DF90CF90BF900C94541756
:1024B000002399F08B2D8F7126960FB6F894DEBF0E
:1024C0000FBECDBFDF91CF911F910F91FF90EF9085
:1024D000DF90CF90BF900C941E1726960FB6F894FD
:1024E000DEBF0FBECDBFDF91CF911F910F91FF9047
:1024F000EF90DF90CF90BF900C9414170023A9F0B9
:10250000222309F4ADCF812F26960FB6F894DEBFB3
:102510000FBECDBFDF91CF911F910F91FF90EF9034
:10252000DF90CF90BF900C94930E222309F4ADCF8F
:10253000812F26960FB6F894DEBF0FBECDBFDF9178
:10254000CF911F910F91FF90EF90DF90CF90BF90B0
:102550000C945B0F4B2D4F70612FC7010E9401023D
:1025600026960FB6F894DEBF0FBECDBFDF91CF9198
:102570001F910F91FF90EF90DF90CF90BF900C9440
:1025800038164B2D4F70612FC70126960FB6F89461
:10259000DEBF0FBECDBFDF91CF911F910F91FF9096
:1025A000EF90DF90CF90BF900C940A0526960FB65F
:1025B000F894DEBF0FBECDBFDF91CF911F910F9179
:1025C000FF90EF90DF90CF90BF9008950E94E018A9
:1025D0000E94F0180E94B5180E940A190E94D11D8D
:1025E0000E94201D80E090E00E948C0D80E090E031
:1025F0000C94A20D0E94D0180C94E6120E942E1882
:10260000292F22952F7030E02C3031054CF42A30E0
:1026100031056CF4225031092230310588F407C0AD
:102620002C30310549F02F30310531F009C0803EA2
:1026300048F0803F29F406C093FB882780F908956D
:1026400080E0089581E00895CF93DF9300D000D01B
:102650001F92CDB7DEB70F900F900F900F900F9095
:10266000DF91CF910895CF93DF9300D000D000D0B9
:10267000CDB7DEB726960FB6F894DEBF0FBECDBF3E
:10268000DF91CF9108951F93CF93DF93C09179018C
:1026900016E080917A01C81799F0D0E01C9FF001F4
:1026A0001D9FF00D1124E558FE4F4081518162813C
:1026B0007381848195810E9433132196C770E9CF7D
:1026C000DF91CF911F9108954091AB015091AC01E2
:1026D0006091AD017091AE018091AF019091B00118
:1026E0000C9433138091B00182958F7009F054C01F
:1026F0008091AD01882309F44FC080917901A091A8
:102700007A016091AB017091AC014091AE015091A2
:10271000AF01B6E08A1709F43FC090E041155105BA
:10272000C1F17F3F11F46F3FA1F1B89FF001B99F54
:10273000F00D1124E558FE4F218172132AC020812B
:10274000621327C02281211124C0238134812417E0
:10275000350710F421503109241B350B283C310575
:10276000C0F42091B0012F7020612093B00126E0C9
:10277000289FF001299FF00D1124E058FE4F808121
:102780008F70806180838BEA91E00E94B80F0C9477
:10279000431301968770BECF0895CF92DF92EF92D8
:1027A000FF920F931F93CF93DF93CDB7DEB762975E
:1027B0000FB6F894DEBF0FBECDBF8C0185E0F801E7
:1027C000DE011D9601900D928A95E1F7D8014C919A
:1027D00011965C91119712966C9112971396CD9069
:1027E000DC9014973091AB017091AC018091AE01F7
:1027F0009091AF01009709F46BC17F3F19F43F3FFF
:1028000009F466C1E090AD01EE2009F4C0C020914A
:10281000B001C816D90628F0F601E81BF90BCF0164
:1028200004C0809590958C0D9D1DFF24F394883CE9
:10283000910578F0F12C207F09F0C6C07C2DD98A53
:10284000C88A89890E9424138BEA91E00E94B80FFC
:10285000B1C0822F807F09F046C0751314C03413B5
:1028600012C0611110C02F7020612093B0010E942E
:1028700064138BEA91E00E94B80F8091B001D801F7
:1028800015968C932EC0CD2819F15F3F11F44F3F60
:10289000F9F0F62E61111CC08091790120917A0126
:1028A00036E0821709F45AC090E0389FF001399F52
:1028B000F00D1124E558FE4F7181571306C0708149
:1028C000471303C07281711103C001968770E9CF6D
:1028D000F62E662309F418C18091B00181608093BF
:1028E000B001F12C11C1751308C0341306C0611179
:1028F00004C08091B001D801C3C04D875E878D852B
:102900009E856A8B0E94FE126A898823E1F1662304
:10291000D1F12091B001822F82958F7090E00297C3
:1029200074F08091AB019091AC0198878F831986E8
:10293000DB86CA862C87CE0107960E94B80F86E0F8
:10294000F801ABEAB1E001900D928A95E1F70E949F
:1029500072130E946413FF24F394D6C04D875E87E0
:102960008D859E850E942E18292F22952F7030E08C
:10297000223031050CF0BCC09F7009F0B6C0805EFB
:10298000883008F4C1C0C8010E94B80FE4CFC8164F
:10299000D90608F453C0F601E81BF90BCF01883CB7
:1029A000910508F450C0F12C7C2DD98AC88A8989F8
:1029B0000E942413EBEAF1E086E0DF011D928A9584
:1029C000E9F70E946413A0C0751314C0341312C039
:1029D000611110C08091B001F8018583C8010E9487
:1029E000B80F86E0EBEAF1E0DF011D928A95E9F786
:1029F000FE2C8AC04D875E878D859E856A8B0E94DE
:102A0000FE126A89882309F4BECF662309F4BBCF7E
:102A10002091B001822F82958F7090E002970CF484
:102A20008ECF8091AB019091AC019A8389831B82F8
:102A3000DD82CC822E83CE0101967FCF809590954A
:102A40008C0D9D1DACCFF62E662309F49CCF75131B
:102A50002EC034132CC02091B00120FD1FC0822F46
:102A600082958F70D9F0D80115962C9315978F30D9
:102A700049F08F5F982F9295907F822F8F70892BCE
:102A800015968C93C8010E94B80F86E0F801ABEA56
:102A9000B1E001900D928A95E1F793CF86E0F801BD
:102AA000ABEAB1E001900D928A95E1F72DC04D8718
:102AB0005E878D859E850E94FE12811140CF809198
:102AC000B00181608093B001C8010E94B80F1CC0A2
:102AD000662309F458CF4D875E878D859E850E94B9
:102AE000FE12882309F44FCF2ACF811148CF0CC0A2
:102AF000243031050CF047CF9F7009F440CFF80126
:102B00009581907F09F03BCF8F2D62960FB6F89498
:102B1000DEBF0FBECDBFDF91CF911F910F91FF9010
:102B2000EF90DF90CF9008951F93CF93DF93CDB7B1
:102B3000DEB72C970FB6F894DEBF0FBECDBF4F8324
:102B4000588769877A878B879C87CE0107960E9472
:102B5000CD13882369F08F8198852A853B85232BA7
:102B6000F1F19F3F09F063C08F3F09F060C037C0AB
:102B700086E0FE013796DE01119601900D928A954E
:102B8000E1F76F817885EA85FB85309741F17F3FDA
:102B900011F46F3F21F120917A0130E0C9010196D3
:102BA000877099274091790150E08417950709F4BF
:102BB00047C069837A83FD83EC8396E0929FD001BE
:102BC000939FB00D1124A558BE4FFE013196019080
:102BD0000D929A95E1F780937A010E94431316E0D3
:102BE0008091790190917A018917C1F1189FC001F4
:102BF000112485589E4F0E94CD13882379F1E091CE
:102C000079011E9FF0011124E558FE4F408151814A
:102C100062817381848195810E943313809179014F
:102C200090E001968770992780937901D9CF4F81E1
:102C3000588569857A858B859C850E943313CFCF13
:102C40000E94FA1210927A0110927901EBEAF1E0F7
:102C500086E0DF011D928A95E9F7C1CF2C960FB669
:102C6000F894DEBF0FBECDBFDF91CF911F910895C5
:102C7000EF92FF920F931F93CF93DF938C01892BD9
:102C800009F46CC0F12CEE24E394E8012196F801DC
:102C90008491843740F4843008F051C0813081F051
:102CA000823019F15BC0853709F444C0A8F19CE774
:102CB000980F903708F052C08F770E945B0F41C089
:102CC0000E5F1F4FFE01C49180E28C0F883048F4E4
:102CD000C7708E2D01C0880FCA95EAF70E94E318CD
:102CE00014C08C2F0E94930E2DC00E5F1F4FFE014B
:102CF000C49180E28C0F883058F4C7708E2D01C0CB
:102D0000880FCA95EAF70E94E9180E940A191AC0AA
:102D10008C2F0E945B0F16C00E5F1F4FFE01C491E7
:102D2000CC2381F08FE99FE00197F1F700C000000C
:102D3000C150F6CF0E5F1F4FFE01F49003C00E94FA
:102D4000930E8E018F2D882309F49FCFEFE9FFE0CA
:102D50003197F1F700C000008150F5CFDF91CF919E
:102D60001F910F91FF90EF90089508956093B50122
:102D70007093B6018093B7019093B8010C94E6125A
:102D80000F931F930091B5011091B6012091B701E7
:102D90003091B801DC01CB01802B912BA22BB32BFE
:102DA0008093B5019093B601A093B701B093B80199
:102DB0001F910F910C94E6120F931F930091B50190
:102DC0001091B6012091B7013091B801DC01CB011F
:102DD00080239123A223B3238093B5019093B6015E
:102DE000A093B701B093B8011F910F910C94E61214
:102DF0000F931F930091B5011091B6012091B70177
:102E00003091B801DC01CB0180279127A227B3279D
:102E10008093B5019093B601A093B701B093B80128
:102E20001F910F910C94E6121092B1011092B20111
:102E30001092B3011092B4010C94E61241E050E0FC
:102E400060E070E004C0440F551F661F771F8A952D
:102E5000D2F74093B1015093B2016093B3017093E4
:102E6000B4010C94E61241E050E060E070E004C070
:102E7000440F551F661F771F8A95D2F78091B101C5
:102E80009091B201A091B301B091B401482B592B9C
:102E90006A2B7B2B4093B1015093B2016093B30135
:102EA0007093B4010C94E61241E050E060E070E0F1
:102EB00004C0440F551F661F771F8A95D2F74095AF
:102EC0005095609570958091B1019091B201A0915B
:102ED000B301B091B401482359236A237B23409363
:102EE000B1015093B2016093B3017093B4010C949B
:102EF000E61241E050E060E070E004C0440F551F6E
:102F0000661F771F8A95D2F78091B1019091B20127
:102F1000A091B301B091B401482759276A277B27B4
:102F20004093B1015093B2016093B3017093B40127
:102F30000C94E6120F931F930091B1011091B2010E
:102F40002091B3013091B401DC01CB01802B912B96
:102F5000A22BB32B8093B1019093B201A093B30144
:102F6000B093B4011F910F910C94E6120F931F932D
:102F70000091B1011091B2012091B3013091B401DF
:102F8000DC01CB0180239123A223B3238093B101E1
:102F90009093B201A093B301B093B4011F910F912C
:102FA0000C94E6120F931F930091B1011091B2019E
:102FB0002091B3013091B401DC01CB01802791272E
:102FC000A227B3278093B1019093B201A093B301DC
:102FD000B093B4011F910F910C94E6120895CF9213
:102FE000DF92EF92FF920F931F93CF93DF938C01A9
:102FF000C090B501D090B601E090B701F090B80153
:103000008091B1019091B201A091B301B091B4014E
:10301000C82AD92AEA2AFB2ACFE1D0E0D701C60183
:103020000C2E04C0B695A795979587950A94D2F76C
:1030300080FF06C0B8018C2F0E942D05019721F456
:10304000219760F780E001C08C2FDF91CF911F9115
:103050000F91FF90EF90DF90CF900895CF93DF9383
:10306000EC010E94EF17BE010E942D05DF91CF9168
:103070000895CB010E942E18089590910C01992378
:1030800021F090910D01911109C020910E01309114
:103090000F01F90132969FEF40E01FC0982F9695DF
:1030A000969596959F3050F5E0910E01F0910F01A5
:1030B000E90FF11D877021E030E0A90102C0440F43
:1030C000551F8A95E2F7CA019181892B8183089562
:1030D0009F3F39F04F5F4E3041F051915813F8CF78
:1030E0000DC05111F7CF942FF5CF9F3F39F0F90163
:1030F000E90FF11D97FDFA95828308950895909147
:103100000C01992321F090910D01911109C020919A
:103110000E0130910F01F9013296205F3F4F1FC021
:10312000982F9695969596959F30F0F4E0910E0124
:10313000F0910F01E90FF11D877021E030E0A90146
:1031400002C0440F551F8A95E2F7CA01809591810C
:103150008923818308953196E217F30729F090813E
:103160009813F9CF1082F7CF089581E090E0E091B5
:103170000E01F0910F01E80FF91F108201968031C6
:103180009105A9F708959091CC01892B8093CC01EA
:10319000089580959091CC0189238093CC01089566
:1031A0001092CC0108959091CB01892B8093CB0193
:1031B000089580959091CB0189238093CB01089548
:1031C0001092CB0108959091CA01892B8093CA0176
:1031D000089580959091CA0189238093CA0108952A
:1031E0001092CA0108958093B90108951092B9010F
:1031F000089580910E0190910F01FC0131969C0180
:10320000205F3F4F80E0919191118F5FE217F307AC
:10321000D1F70895E0910E01F0910F018091CC015A
:103220008083E0910E01F0910F0190818091CB019C
:10323000892B8083E0910E01F0910F0190818091A4
:10324000CA01892B80838091B901882361F0E091C4
:103250000E01F0910F019081892B80830E94F91853
:1032600081111092B90180910E0190910F010C947F
:10327000760D8091E601843021F11092CE0120E498
:1032800088E190E00FB6F894A895809360000FBE97
:103290002093600080E00E94630683B7817F846092
:1032A00083BF83B7816083BF7894889583B78E7F0F
:1032B00083BF88E10FB6F89480936000109260009D
:1032C0000FBE089508950895CF930E9462190E9439
:1032D00056030E946319C0E08C2F0E9444048111A0
:1032E00004C0CF5FCE30C1F701C081E0CF91089517
:1032F0000E94FA120E946A0D0C94630682E084BD5B
:1033000093E095BD9AEF97BD80936E0008952FB717
:10331000F8948091CF019091D001A091D101B0910A
:10332000D2012FBF0895CF92DF92EF92FF920F93B9
:103330001F932FB7F8944091CF015091D001609125
:10334000D1017091D2012FBF6A017B01EE24FF24CD
:103350008C0120E030E0C016D106E206F30610F43E
:10336000415051099A01281B390BC9011F910F9136
:10337000FF90EF90DF90CF9008951F920F920FB6BD
:103380000F9211248F939F93AF93BF938091CF019E
:103390009091D001A091D101B091D2010196A11DCF
:1033A000B11D8093CF019093D001A093D101B09330
:1033B000D201BF91AF919F918F910F900FBE0F904F
:1033C0001F9018950E94670AF8942FEF87EA91E6FC
:1033D000215080409040E1F700C0000087E090EB72
:1033E000DC018093EF019093F001A093F101B09381
:1033F000F2019CE088E10FB6F894A89580936000F4
:103400000FBE90936000FFCFEF92FF920F931F9338
:10341000CF93DF93D82FC0E08C2F0E94440400E0AC
:1034200010E0E82EF12CC701002E02C0959587957B
:103430000A94E2F780FD06C00F5F1F4F06301105AA
:1034400091F709C0602F7C2F80E00E940B05D813F4
:10345000F3CF81E004C0CF5FCE30F1F680E0DF91A2
:10346000CF911F910F91FF90EF900895CF93C82FA8
:103470008CE20E94041A882321F08C2FCF910C94A7
:10348000041A80E0CF910895CF930E948B1B811185
:1034900002C00E94711BC5E6C15049F00E9456034C
:1034A0008FE39CE90197F1F700C00000F5CF89E2B6
:1034B0000E94361A811113C18AE20E94361A8111C4
:1034C0000E94711B85E00E94361A81110E94E21948
:1034D0000E94961B8093CD0187E00E94361A8823B4
:1034E000A9F18BE10E94361A882351F08091CD0119
:1034F00081FB222720F991E0922790FB81F90EC0F1
:103500008EE00E94361A882361F08091CD0182FB03
:10351000222720F991E0922790FB82F98093CD0138
:1035200015C080E10E94361A9091CD01882341F0A8
:1035300093FB222720F981E0822780FB93F904C0C6
:10354000892F809580FB90F99093CD018091CD01DA
:103550000E949A1B0E94A81B8093E00180EE0E94AB
:10356000361A882341F08091E001982F909590FBC6
:1035700080F98093E00189E30E94361A882359F08C
:103580008091E00181FB222720F991E0922790FBB6
:1035900081F98093E00182EE0E94361A882359F067
:1035A0008091E00182FB222720F991E0922790FB95
:1035B00082F98093E00186EE0E94361A882359F042
:1035C0008091E00183FB222720F991E0922790FB74
:1035D00083F98093E00183EE0E94361A882359F024
:1035E0008091E00184FB222720F991E0922790FB53
:1035F00084F98093E00185E30E94361A882359F00C
:103600008091E00185FB222720F991E0922790FB31
:1036100085F98093E00181E30E94361A882359F0EE
:103620008091E00186FB222720F991E0922790FB10
:1036300086F98093E00181E10E94361A882359F0CF
:103640008091E00187FB222720F991E0922790FBEF
:1036500087F98093E0018091E0010E94AC1B80918A
:10366000E00187FB882780F980930D0187E20E94A3
:10367000361AC82F8EE10E94361A8111C2608FE17E
:103680000E94361A8111C46080E20E94361A8111AC
:10369000C86081E20E94361A8111C06182E20E94F4
:1036A000361A8111C06283E20E94361A8111C06409
:1036B00084E20E94361A882311F0C06802C0CC232D
:1036C00029F08C2F0E94A31B6C2F03C00E949F1B0C
:1036D000682F70E080E090E0CF910C94B616CF9107
:1036E00008956DEE7EEF80E090E00E94DD2160E0C5
:1036F00082E090E00E94CF2160E083E090E00E94B1
:10370000CF2160E084E090E00E94CF2160E085E07E
:1037100090E00C94CF2180E090E00E94C92121E04C
:103720008D3E9E4F09F020E0822F089582E090E0C8
:103730000C94C121682F82E090E00C94CF2183E0AB
:1037400090E00C94C121682F83E090E00C94CF218D
:1037500084E090E00C94C121682F84E090E00C9408
:10376000CF218091D50180FF0BC06091130185E0CE
:10377000689FB001112475956795759567952BC065
:1037800081FF09C06091130185E0689FB001112499
:103790007595679520C082FF07C06091130185E091
:1037A000689FB001112417C09091D6019923D1F0E0
:1037B00060911201961788F72091130185E0289FE8
:1037C00090011124929FA001939F500D112470E04D
:1037D000CA010E9493216038710540F4611571059A
:1037E00039F002C065E070E0862F08958FE70895F4
:1037F00081E008958091D50180FF08C0609111019A
:1038000070E0759567957595679521C081FF06C035
:103810006091110170E07595679519C082FF04C031
:103820006091110170E010C09091D6019923C1F010
:10383000609110019617A0F780911101899FC00136
:10384000112470E00E9493216038710528F46115FD
:10385000710521F0862F08958FE7089581E008957E
:1038600061E070E0F4CF803F21F40E94B11B8195AC
:1038700004C0813F29F40E94B11B8093D9010895AF
:10388000823F21F40E94B11B819504C0833F29F43B
:103890000E94B11B8093D8010895893F19F40E94BA
:1038A000FA1B05C08A3F31F40E94FA1B8195809370
:1038B000DA0108958B3F21F40E94FA1B819504C020
:1038C0008C3F29F40E94FA1B8093DB010895843F0A
:1038D00021F48091D701816017C0853F21F4809148
:1038E000D701826011C0863F21F48091D7018460A6
:1038F0000BC0873F21F48091D701886005C0883FC5
:1039000031F48091D70180618093D70108958D3F74
:1039100021F48091D50181600BC08E3F21F480910C
:10392000D501826005C08F3F29F48091D501846064
:103930008093D5010895803F39F48091D90187FFA4
:103940006CC01092D90169C0813F29F48091D901DE
:103950001816BCF362C09091D801823F29F497FFFA
:103960005CC01092D80159C0833F19F41916CCF3EA
:1039700054C0893F41F48091DA0118160CF04DC013
:103980001092DA014AC08A3F29F48091DA0187FF58
:1039900044C0F6CF8B3F39F48091DB0187FF3DC0F7
:1039A0001092DB013AC08C3F29F48091DB0118169C
:1039B000BCF333C0843F21F48091D7018E7F17C0C0
:1039C000853F21F48091D7018D7F11C0863F21F47E
:1039D0008091D7018B7F0BC0873F21F48091D70165
:1039E000877F05C0883F31F48091D7018F7E809317
:1039F000D70113C08D3F21F48091D5018E7F0BC07C
:103A00008E3F21F48091D5018D7F05C08F3F29F431
:103A10008091D5018B7F8093D5018091D801811150
:103A20000EC08091D90181110AC08091DA01811103
:103A300006C08091DB01811102C01092D601089569
:103A400087ED91E00E94810D0E9487199093D40127
:103A50008093D30108951F93CF93DF938091D30177
:103A60009091D4010E949319AC019091D6019923B1
:103A700021F02091140130E006C0209115018AE068
:103A8000289F900111244217530708F486C08091A3
:103A9000D801C091D901D091DA011091DB018111D7
:103AA00007C0C11176C0D11174C0111172C075C0A8
:103AB0009F3F19F09F5F9093D601181624F40E943F
:103AC000B11B8093D8018091D80187FF05C00E9467
:103AD000B11B81958093D8011C1624F40E94B11B60
:103AE0008093D9018091D90187FF05C00E94B11B45
:103AF00081958093D9016091D801662339F1C091F5
:103B0000D901CC2319F1772767FD7095872F972F5F
:103B10000E94A42023E333E343E35FE30E940821F0
:103B20000E9471206093D8016C2F772767FD7095F4
:103B3000872F972F0E94A42023E333E343E35FE31F
:103B40000E9408210E9471206093D9011D1624F45F
:103B50000E94FA1B8093DA018091DA0187FF05C089
:103B60000E94FA1B81958093DA01111624F40E94B9
:103B7000FA1B8093DB018091DB0187FF05C00E9467
:103B8000FA1B81958093DB01DF91CF911F910C94FB
:103B9000201D9F3F09F08ECF96CFDF91CF911F91CF
:103BA0000895E7EDF1E085E0DF011D928A95E9F7E0
:103BB0001092D6011092D5010895833081F128F436
:103BC000813059F08230D1F00895853009F449C030
:103BD000B8F1863009F456C0089580911501262F5A
:103BE00030E0280F311D2F3F310524F4680F60931A
:103BF000150108958FEF80931501089580911401A8
:103C0000262F30E0280F311D2F3F310524F4680F97
:103C10006093140108958FEF8093140108958091AB
:103C20001301262F30E0280F311D2F3F310524F4DA
:103C3000680F6093130108958FEF80931301089527
:103C400080911201262F30E0280F311D2F3F3105C2
:103C500024F4680F6093120108958FEF809312018E
:103C6000089580911101262F30E0280F311D2F3F3C
:103C7000310524F4680F6093110108958FEF80934C
:103C80001101089580911001262F30E0280F311D79
:103C90002F3F310524F4680F6093100108958FEFD2
:103CA000809310010895833011F128F4813049F098
:103CB000823091F00895853081F120F18630C1F194
:103CC000089580911501681720F4861B80931501D3
:103CD000089510921501089580911401681720F439
:103CE000861B809314010895109214010895809109
:103CF0001301681720F4861B809313010895109216
:103D00001301089580911201681720F4861B809397
:103D100012010895109212010895809111016817FF
:103D200020F4861B809311010895109211010895CB
:103D300080911001681720F4861B8093100108956C
:103D40001092100108950F931F938D3109F46AC0EA
:103D500008F03FC08E3009F484C0C0F4873009F405
:103D60006DC068F4863009F0B5C08091CD01817FC7
:103D70008E7F8093CD0181E08093DD01ACC08830DF
:103D800009F457C08B3009F46AC0A4C0863109F425
:103D900066C078F4803109F477C0813109F09AC0A7
:103DA0000E94FA1290910D0181E0892780930D0104
:103DB00056C0893109F453C08B3109F08BC0809112
:103DC000CD0181FB222720F991E0922790FB81F918
:103DD00051C0853309F475C048F4873209F471C0C5
:103DE00008F45EC0893209F46CC074C0833430F4C6
:103DF0008A3308F053C0883391F16CC0833409F4DE
:103E000060C0883409F066C00E94FA120FEF13ED0B
:103E100020E3015010402040E1F700C000000E9464
:103E2000E2191DC00E942B200E946A0D0E946306A9
:103E300016C00E94961B0E94A81B11C09091CD0134
:103E4000892F8095817080FB90F929F096609860A9
:103E50009093CD0140C0997F977F9093CD0181E0F1
:103E60003AC08091CD0182FB222720F991E0922770
:103E700090FB82F98093CD01992389F38091CD0144
:103E800081608093CD01EBCF8091CD0183FB222710
:103E900020F991E0922790FB83F9ECCF895301C080
:103EA0008D5141E050E060E070E08A019B0104C068
:103EB000000F111F221F331F8A95D2F7C901B801C5
:103EC00004C061E070E080E090E00E94B6160E94BD
:103ED000FA12C5CF80E01F910F91089580E00895F8
:103EE00080E00895CF93C82F8091DD01813079F073
:103EF00018F08230E9F187C0E0910E01F0910F01D6
:103F00008081813169F0823209F07FC009C0E0917F
:103F10000E01F0910F018081813111F0823261F444
:103F20008C2F0E946E1F811104C08C2F0E94A31E33
:103F30001DC081E090E01AC08C2F0E94701F81117B
:103F400014C0C43179F048F4CB3079F0C03109F0B5
:103F500060C082E08093DD0108C0C93219F0C83327
:103F600021F057C01092DD0154C081E0817053C030
:103F7000C93289F118F5C43171F1A8F4C73009F0DC
:103F800046C08AE08093150194E19093140193E078
:103F9000909313018093120188E08093110188E2CD
:103FA0008093100134C0CE51C63088F5EC2FF0E07C
:103FB000E65DFE4F80818093DC0129C0CE34E9F0BC
:103FC00020F4CB3421F56AE013C0C13579F0C23555
:103FD000F1F461E00DC08091DC01882319F01092AA
:103FE000DC0115C081E08093DD0115C061E006C0F1
:103FF0008091DC010E94DD1D0AC06AE08091DC0135
:104000000E94531E04C01092DD0180E004C081E0D4
:1040100002C080E0ABCFCF910895E1E8F0E080816D
:10402000886080838081816080838FB7F89493E07B
:104030009093890090ED909388008FBF0895EFE6EC
:10404000F0E08081826080830895EFE6F0E0808177
:104050008D7F80830895EFE6F0E0908182E08927EC
:10406000808308951F920F920FB60F9211242F9301
:104070003F934F935F936F937F938F939F93AF93F0
:10408000BF93EF93FF938091DE019091DF01019642
:104090009093DF018093DE01811103C082E00E94D2
:1040A0006306E091DF01E695E695F0E0EA5CFC4FFF
:1040B000E4918091DE018E1303C080E00E946306CC
:1040C000FF91EF91BF91AF919F918F917F916F91F0
:1040D0005F914F913F912F910F900FBE0F901F90C6
:1040E000189504D06894B1118DC0089570D088F0EF
:1040F0009F5790F0B92F9927B751A0F0D1F0660FD4
:10410000771F881F991F1AF0BA95C9F712C0B130EE
:1041100081F077D0B1E0089574C0672F782F882799
:10412000B85F39F0B93FCCF3869577956795B3952D
:10413000D9F73EF490958095709561957F4F8F4F9C
:104140009F4F0895E89409C097FB3EF490958095A1
:10415000709561957F4F8F4F9F4F9923A9F0F92F4D
:1041600096E9BB279395F695879577956795B795CB
:10417000F111F8CFFAF4BB0F11F460FF1BC06F5FB1
:104180007F4F8F4F9F4F16C0882311F096E911C0C3
:10419000772321F09EE8872F762F05C0662371F0E4
:1041A00096E8862F70E060E02AF09A95660F771FF8
:1041B000881FDAF7880F9695879597F9089557FD28
:1041C0009058440F551F59F05F3F71F04795880F85
:1041D00097FB991F61F09F3F79F08795089512161C
:1041E00013061406551FF2CF4695F1DF08C01616C8
:1041F00017061806991FF1CF869571056105089479
:104200000895E894BB2766277727CB0197F908958F
:104210000BD078C069D028F06ED018F0952309F043
:104220005AC05FC01124EECFCADFA0F3959FD1F32F
:10423000950F50E0551F629FF001729FBB27F00D54
:10424000B11D639FAA27F00DB11DAA1F649F6627A9
:10425000B00DA11D661F829F2227B00DA11D621FF8
:10426000739FB00DA11D621F839FA00D611D221FB2
:10427000749F3327A00D611D231F849F600D211D96
:10428000822F762F6A2F11249F5750408AF0E1F039
:1042900088234AF0EE0FFF1FBB1F661F771F881F82
:1042A00091505040A9F79E3F510570F014C0AACF1D
:1042B0005F3FECF3983EDCF3869577956795B7956D
:1042C000F795E7959F5FC1F7FE2B880F911D969597
:1042D000879597F9089597F99F6780E870E060E007
:1042E00008959FEF80EC089500240A94161617068F
:1042F00018060906089500240A94121613061406D7
:1043000005060895092E0394000C11F4882352F039
:10431000BB0F40F4BF2B11F460FF04C06F5F7F4FF1
:104320008F4F9F4F089597FB072E16F4009407D0E8
:1043300077FD09D00E94AD2107FC05D03EF4909591
:1043400081959F4F0895709561957F4F0895EE0F69
:10435000FF1F0590F491E02D0994AA1BBB1B51E1AE
:1043600007C0AA1FBB1FA617B70710F0A61BB70BE5
:10437000881F991F5A95A9F780959095BC01CD018A
:104380000895F999FECF92BD81BDF89A992780B51D
:104390000895A8E1B0E042E050E00C94E421262F1B
:1043A000F999FECF1FBA92BD81BD20BD0FB6F8941A
:1043B000FA9AF99A0FBE019608950E94CF21272FED
:1043C0000C94D021DC01CB01FC01F999FECF06C091
:1043D000F2BDE1BDF89A319600B40D9241505040C3
:0843E000B8F70895F894FFCF2F
:1043E80020026506F306D0069C0668060101BA019C
:1043F80028080A03140A3F4D3639F702AA02740244
:104408003B02CE01E701000219020102030405067E
:044418000708090088
:00000001FF
